:020000040800F2
:1000000058250020390200080D1000084B03000895
:100010000910000845030008F11200080000000064
:10002000000000000000000000000000A101000826
:100030004903000800000000E50100082D11000838
:10004000530200085302000853020008530200083C
:10005000530200085302000853020008530200082C
:10006000530200085302000853020008530200081C
:10007000530200085302000853020008530200080C
:1000800053020008530200085302000853020008FC
:1000900053020008530200085302000853020008EC
:1000A00053020008530200085302000853020008DC
:1000B00053020008530200085302000853020008CC
:1000C00053020008530200085302000853020008BC
:1000D00053020008530200085302000853020008AC
:1000E000530200085302000853020008530200089C
:1000F000530200085302000853020008530200088C
:10010000530200085302000853020008530200087B
:10011000530200085302000853020008530200086B
:10012000530200085302000853020008530200085B
:10013000530200085302000853020008530200084B
:10014000530200085302000853020008530200083B
:10015000530200085302000853020008530200082B
:10016000530200085302000853020008530200081B
:100170005302000853020008530200080000000068
:100180005302000853020008DFF810D000F0C8F84E
:1001900000480047FD130008AFF3008058250020F9
:1001A000224B19680868B0E8F00F80F30988BFF3A4
:1001B0006F8F4FF0000080F311884EF00D0E7047E6
:1001C0000000000006480068006880F3088862B6F6
:1001D00061B6BFF34F8FBFF36F8F00DF00BF00BF6B
:1001E00008ED00E0EFF30980BFF36F8F0F4B1A6843
:1001F00020E9F00F106008B54FF0BF0080F31188C0
:10020000BFF34F8FBFF36F8F01F0EEFD4FF0000093
:1002100080F31188BDE8084019680868B0E8F00F5D
:1002200080F30988BFF36F8F704700BF1000002074
:10023000EFF30580704700000648804706480047F6
:10024000FEE7FEE7FEE7FEE7FEE7FEE7FEE7FEE786
:10025000FEE7FEE7DD120008890100082DE9F05FE6
:100260000546002092469B46884606468146402425
:100270001BE0284641464746224600F041F85346D7
:100280005A46C01A914110D311461846224600F032
:1002900028F82D1A67EB01084F462246012000215D
:1002A00000F01FF817EB00094E41201EA4F10104D5
:1002B000DFDC484631462A464346BDE8F09FD2B2CD
:1002C00001E000F8012B491EFBD270470022F6E73F
:1002D00010B513460A4604461946FFF7F0FF2046BC
:1002E00010BD202A04DB203A00FA02F100207047FA
:1002F0009140C2F1200320FA03F319439040704764
:10030000202A04DB203A21FA02F00021704721FA6A
:1003100002F3D040C2F120029140084319467047D1
:10032000064C074D06E0E06840F0010394E8070042
:1003300098471034AC42F6D3FFF72AFF0822000892
:100340002822000800BFFEE7704700BFFEE700005C
:1003500008B5054909680143034A11601146096857
:100360000140009100BF08BD30380240F0B50246A0
:100370000B4600240021186890FAA0F0B0FA80F42F
:100380008AE00125A540186800EA050100297DD012
:100390005868012802D0586802281CD198689568CE
:1003A00091FAA1F6B6FA86F677000326BE40B54369
:1003B00091FAA1F6B6FA86F6760000FA06F635430B
:1003C000956000BFD86855688D4301FB00F6354342
:1003D000556000BF00BF1869D56891FAA1F6B6FA5A
:1003E00086F677000326BE40B54391FAA1F6B6FA29
:1003F00086F6760000FA06F63543D56000BF5868E9
:10040000022831D191FAA1F0B0FA80F0082814D274
:100410005869156A91FAA1F6B6FA86F6B7000F2662
:10042000BE40B54391FAA1F6B6FA86F6B60000FAD8
:1004300006F63543156200BF16E05869556A0E0A84
:1004400096FAA6F6B6FA86F6B7000F26BE40B54372
:100450000E0A96FAA6F6B6FA86F6B60000FA06F680
:100460003543556200BF00BF5868156891FAA1F680
:10047000B6FA86F677000326BE40B54391FAA1F698
:10048000B6FA86F6760000FA06F600E003E0354399
:10049000156000BF00BF641C1868E04000287FF4AE
:1004A00070AFF0BD4FF47A71B0FBF1F2521E4FF015
:1004B000E0235A6100229A6105221A6100BF704749
:1004C00002480068C0F30020704700000070004040
:1004D00010B5044600F0D0FD2060206800F098FDC3
:1004E0006060606800F0A4FDA060606800F0B2FD8C
:1004F000E06010BD02480068C0F38810704700003B
:1005000004380240F0B5059C04F0F006360404F00F
:100510000F0746EA074646EA413603F0F0073F0276
:1005200003F00F0C47EA0C273E4302F0F00702F0FD
:100530000F0C47EA0C0746EA07054668024F3E40A3
:100540002E434660F0BD0000C00000FF2DE9F84FCB
:1005500006460D46144601274DB9607800F010009C
:10056000102804D1607800F0EF000A30607005B9FF
:1005700000E000BF304600F058F8304600F05DF86B
:10058000012848D045B1E07800906378A2782178BE
:100590003046FFF7B7FF31E0E0780A21B0FBF1F217
:1005A00001FB1200E1780A22B1FBF2F140EA0110EE
:1005B00000F0FF0860781146B0FBF1F201FB120079
:1005C00061780A22B1FBF2F140EA011000F0FF0964
:1005D000A0781146B0FBF1F201FB1200A1780A22CB
:1005E000B1FBF2F140EA011000F0FF0ACDF8008003
:1005F00021784B4652463046FFF784FF304600F0E4
:1006000010F8304600F07BF820B9304600F00EF9C3
:10061000074600E00027304600F00CF83846BDE8F9
:10062000F88F6FF08001C1607047CA214162532189
:1006300041627047FF2141627047F8B504464FF4AC
:100640007A70009000250026204600F04EF8D0B9C0
:1006500000BF681EE06000BF204600F046F8064676
:100660000DE000F00BF9012802D10098401E009027
:10067000204600F03AF80646009800B90125009897
:1006800008B1012EEDD12846F8BD0146886800F07A
:100690004000704770B504460D4601262046FFF71E
:1006A000C4FF2046FFF7C9FF012819D02868A168B8
:1006B00021F040010143A16000BFA86821696FF3E8
:1006C0000E010143216100BF6868216921F4FE0128
:1006D00041EA0041216100BF2046FFF7A2FF00264A
:1006E0002046FFF7A7FF304670BD0146C868C0F33B
:1006F000801070470146C868C0F34010704701463B
:100700008868C0F340107047F0B5059C02F0F00611
:10071000360402F00F0746EA07460E4303F0F007DF
:100720003F0203F00F0C47EA0C273E4304F0F007AA
:1007300004F00F0C47EA0C0746EA07050668024F6B
:100740003E402E430660F0BD808080FF2DE9F84FCB
:1007500006460D461446012745B93046FFF795FF7A
:1007600000B102E00020206000BF08E03046FFF743
:100770008CFF00B102E00020206000BF00BF3046C7
:10078000FFF753FF3046FFF758FF012848D045B127
:10079000A07900906379227930462168FFF7B4FF91
:1007A00031E0A0790A21B0FBF1F201FB1200A1793E
:1007B0000A22B1FBF2F140EA011000F0FF08607973
:1007C0001146B0FBF1F201FB120061790A22B1FB84
:1007D000F2F140EA011000F0FF0920791146B0FB68
:1007E000F1F201FB120021790A22B1FBF2F140EA99
:1007F000011000F0FF0ACDF800804B46524630460B
:100800002168FFF781FF3046FFF70BFF3046FFF707
:1008100076FF20B9304600F009F8074600E00027CF
:100820003046FFF707FF3846BDE8F88FF8B50446B5
:100830004FF47A7000900025002600BFE06800F0B9
:10084000800060F0A000E06000BF2046FFF752FF8C
:1008500006460DE000F012F8012802D10098401E73
:1008600000902046FFF746FF0646009800B9012594
:10087000009808B1012EEDD12846F8BD4FF0E020D8
:100880000069C0F3004070470149086070470000EC
:100890000000002010B5024613682C4882420ED09A
:1008A000B2F1804F0BD02A48824208D029488242B8
:1008B00005D02948824202D02848824204D123F040
:1008C00070004C6840EA04032048824220D0B2F114
:1008D000804F1DD01E4882421AD01E48824217D037
:1008E0001D48824214D01D48824211D01C488242C9
:1008F0000ED01C4882420BD01B48824208D01B48B5
:10090000824205D01A48824202D01A48824204D15B
:1009100023F44070CC6840EA040313608868D06216
:1009200000BF0888906200BF0848824202D00B488E
:10093000824203D10869106300BF00BF00BF506945
:1009400040F00100506100BF002010BD00000140D8
:100950000004004000080040000C0040000401407A
:1009600000400140004401400048014000180040A0
:10097000001C0040002000402DE9FF4104460D46C8
:1009800001270026204600F059F8002845D1E968E3
:100990006868084329690843A9690843E16849F27E
:1009A0000C6291430843E060A868216921F440513A
:1009B0000143216100BF6869616921F4407101430D
:1009C000616100BF6846FFF783FD1648844201D18C
:1009D000039E17E01448844201D1029E12E013489E
:1009E000844201D1029E0DE01148844201D1039E50
:1009F00008E01048844201D1029E03E00E48844280
:100A000000D1029E4EB1286838B1002731462046F9
:100A10002B68AA6900F017F800BF384604B0BDE89B
:100A2000F0810000001001400044004000480040F8
:100A300000140140004C0040005000400146C868CE
:100A4000C0F3403070472DE9FC5F06460C469146E6
:100A50001D46B9F5004F68D10220A0FB0570034682
:100A60001920A4FB00A001463A465046FFF7F6FBCA
:100A70006421B0FBF1F04FEA001A0220A0FB0571DF
:100A80000B461920A4FB00B13A465846FFF7E6FB97
:100A900083460220A0FB057003461920A4FB000139
:100AA0003A46CDE90001FFF7D9FB6421B0FBF1F034
:100AB00000EBC00101EB0010ABEB8000322101EB39
:100AC000C0006421B0FBF1F000F0F8000AEB400A2E
:100AD0000220A0FB057003461920A4FB00B13A4692
:100AE0005846FFF7BBFB83460220A0FB0570034678
:100AF0001920A4FB00013A46CDE90001FFF7AEFB47
:100B00006421B0FBF1F000EBC00101EB0010ABEB96
:100B10008000322101EBC0006421B0FBF1F000F055
:100B20000700504480B2B06067E00420A0FB05706D
:100B300003461920A4FB00A001463A465046FFF7A1
:100B40008DFB82460420A0FB05711920A4FB00B098
:100B500084463A460B4658466146FFF77FFB6421C0
:100B6000B0FBF1F000EBC00101EB0010AAEB80003C
:100B7000322101EB00106421B0FBF1F000F0F00A2B
:100B80000420A0FB057003461920A4FB00B0014619
:100B90003A465846FFF762FB6421B0FBF1F00AEBDE
:100BA000001A0420A0FB057003461920A4FB00B125
:100BB0003A465846FFF752FB83460420A0FB0570D7
:100BC00003461920A4FB00013A46CDE90001FFF7D6
:100BD00045FB6421B0FBF1F000EBC00101EB00101C
:100BE000ABEB8000322101EB00106421B0FBF1F08F
:100BF00000F00F00504480B2B060BDE8FC9F0000E0
:100C000000B587B0182101A8FFF760FB1020FFF79F
:100C10009FFB0420FFF79CFB2020FFF799FB80201F
:100C2000FFF796FB0120FFF793FB0220FFF790FBF5
:100C30004020FFF78DFB0820FFF78AFB4FF40050A0
:100C400001042F4A916100BF4FF6FF70019003200D
:100C500002900020059001A92A48FFF787FB4FF476
:100C60000050019001200290002003900490059014
:100C700001A92348FFF77AFB4FF6FF70019003208C
:100C800002900020059001A91F48FFF76FFB41F675
:100C9000FF700190032002900020059001A91848E0
:100CA000FFF764FB49F6FF1001900320029000203B
:100CB000059001A91548FFF759FB4FF6FF70019009
:100CC000032002900020059001A91148FFF74EFB78
:100CD0004FF6FF700190032002900020059001A9BB
:100CE0000C48FFF743FB4FF6FF7001900320029082
:100CF0000020059001A90848FFF738FB07B000BDA8
:100D000000080240001002400014024000000240AF
:100D10000004024000180240000C024010B588B0E8
:100D2000002005900690079003900490029000BF69
:100D30006448006800F44070B0F5807F6AD00024F9
:100D40004FF080505F49303909680140814201D13C
:100D5000012100E0002101290FD04FF080505949B6
:100D6000303909680143574A303A11601146096821
:100D70000140019100BF00BF0124FFF7A1FB012842
:100D80000CD000BF5048006840F480704E490860A5
:100D900000BF00BFFFF794FB0028FBD000BF49480D
:100DA000006840F480304749086000BF00BF084633
:100DB000006820F48030086000BF00BF084600686B
:100DC00040F00400086000BF00BF0846006840F023
:100DD0000100086000BF00BF00BF3A480068C0F3D0
:100DE00040000028F8D04FF480703649096821F49B
:100DF00040710143334A116000BF012C09D1000545
:100E000030493039096881432E4A303A116000BFB9
:100E100000BF00BF00BF2B48006840F400402949D4
:100E2000086000BF002005907F200690FF200790FB
:100E300005A92648FFF72EFC7F202449096921F4E3
:100E4000FE0141EA0041214A116100BFFF20114625
:100E500009696FF30E010143116100BF11460020C3
:100E600001F1500202EB8002136843F2F220834248
:100E700025D000208DF810008DF811008DF812009B
:100E800003AA01211148FFF761FC01208DF8080039
:100E90008DF809008DF80A0000208DF80B0002AAD9
:100EA00001210A48FFF752FB0849002043F2F222D1
:100EB00001F1500303EB80031A6000BF00BF08B0CC
:100EC00010BD000070380240007000400028004053
:100ED00000B587B0142102A8FFF7F8F910201849CF
:100EE00009680143164A11601146096801400191E1
:100EF00000BF00BF42F2CF00ADF808000020039011
:100F00006320049002A90F48FFF7C4FC00BF0D48FE
:100F1000006820F080000B49086000BF002049688D
:100F200021F070010143074A516000BF00BF104625
:100F3000806820F080001146886000BF07B000BDC7
:100F4000403802400010004000B58FB01C2108A8B6
:100F5000FFF7BCF9182102A8FFF7B8F910202749BC
:100F600009680143254A1160114609680140019151
:100F700000BF00BF012021491439096801431F4AFD
:100F8000143A1160114609680140019100BF00BF89
:100F90004FF4C060029002200390032004900020D0
:100FA000059006900720079002A91548FFF7DEF983
:100FB0004FF4E1300890002009900A900B900C202B
:100FC0000C9000200D900E9008A90E48FFF7D4FC5D
:100FD00000BF0C48006920F490400A4908610846A7
:100FE000406920F02A00486100BF00BF0846C06881
:100FF00040F40050C86000BF0FB000BD443802404C
:10100000000002400010014000BFFEE700BFFEE705
:10101000014600BF0448006800F0F0000009034AE0
:10102000125C21FA02F0704708380240D82100080B
:10103000014600BF0548006800F4E050044A02EB96
:101040009020027821FA02F0704700000838024030
:10105000E8210008014600BF0548006800F4604030
:10106000044A02EB5030027821FA02F07047000087
:1010700008380240E821000810B5002400BF0C48E1
:10108000006800F00C0020B1042804D0082809D121
:1010900003E0084C08E0084C06E0082000F00EF8D9
:1010A000044601E0034C00BF00BF204610BD000015
:1010B000083802400024F40000127A002DE9F041C3
:1010C000044600250026002700BF1548006800F4EC
:1010D000800006461EB1B6F5800F04D101E0114D27
:1010E00003E0114D01E00F4D00BF00BF082C14D1EB
:1010F00000BF0B48006800F03F00B5FBF0F8FFF7B9
:10110000F9F908FB00F80648006800F440300121B6
:1011100001EB10404000B8FBF0F73846BDE8F08125
:10112000043802400024F40000127A0010B500BF19
:10113000BF2080F31188BFF34F8FBFF36F8F00BFC5
:1011400000F0BCFE18B14FF080500449086000BFA9
:10115000002080F3118800BF10BD000004ED00E006
:1011600070B505205849096821F007010143564A26
:10117000116000BF00BF00BF5348006800F00700C7
:101180000528F8D14FF480405049096821F4804186
:1011900001434E4A116000BF00BF4D48006840F453
:1011A00080304B49086000BF00BF00BF484800685E
:1011B000C0F340400028F8D000BF4448006840F425
:1011C00080704249086000BF00BF4148703000682D
:1011D00040F004003E497031086000BF00BF08467F
:1011E000006840F00100086000BF00BF00BF384841
:1011F00070300068C0F340000028F7D04FF4800042
:101200000421A822002340EA010444EA8214304D5C
:101210002D1D2D682F4E35402C432D4D2D1D2C603E
:101220002C46246824F440341C432C6000BF00BFCB
:10123000281F006840F08070291F086000BF00BFB1
:1012400000BF23480068C0F340600028F8D000BF0A
:1012500000BF1E484068C0F380300028F8D000204E
:101260001B490831096821F0F0010143184A08328E
:10127000116000BF4FF4A0501146096821F4E051FD
:101280000143116000BF4FF400401146096821F48A
:1012900060410143116000BF02201146096821F03E
:1012A00003010143116000BF00BF00BF08480830C0
:1012B000006800F00C000828F7D10748FFF7F2F8A3
:1012C0000548FFF7E1FA70BD003C024000700040A5
:1012D000003802400080BFFF007A030A034800681C
:1012E00040F47000014908607047000088ED00E09C
:1012F00000BFFEE702E008C8121F08C1002AFAD1A9
:1013000070477047002001E001C1121F002AFBD185
:1013100070470000014601F1100000E0001D026866
:101320001AB9024A12689042F8D370470C000020A4
:1013300010B50648046803E02046FFF7EBFF0446BB
:10134000034800688442F7D310BD00000800002065
:101350000C0000201CB50548012100238022CDE9A6
:10136000001003A1064800F08DFD1CBD0400002004
:10137000627573696E6573735F7461736B000000EF
:10138000B913000810B500F001FD10BD1CB51920FF
:10139000ADF8040001208DF806008DF8070000204C
:1013A0008DF800008DF801008DF802000322DDE9C0
:1013B000001000F0BFFB1CBD00BF002000F008F8CB
:1013C00000F000FC4FF47A7000F0C6FCF5E7000076
:1013D00010B5014669B94FF40050074B5A6920EA2D
:1013E000020302EA000443EA0443034CA36100BF82
:1013F00000E000BF00BF10BD0008024008B54FF478
:1014000080403C49096801433A4A11601146096825
:101410000140009100BF00BF8003111F0968014314
:10142000121F1160114609680140009100BF00BF02
:1014300003200246304B19684FF6FF0319402F4B2B
:101440000B4343EA02212C4B196000BF011F1B68AC
:10145000C3F302200F2400250346C3F1070CBCF19F
:10146000040F02D94FF0040C01E0C3F1070C6746EA
:1014700003F1040CBCF1070F02D24FF0000C01E0A5
:10148000A3F1030C66464FF0010C0CFA07FCACF11B
:10149000010C0CEA040C0CFA06FC4FF0010808FAE7
:1014A00006F8A8F1010808EA05084CEA080200BF9E
:1014B000002904DB1007030E1148435407E010070E
:1014C000040E0D480C3001F00F031B1FC45400BF65
:1014D000FFF746FEFFF794FBFFF7FAFCFFF71EFC51
:1014E000FFF732FDFFF752FFFFF734FFFFF74AFF28
:1014F00000BFFEE7443802400CED00E00000FA05B2
:1015000000E400E02DE9F04705460E46294807684B
:101510002948D0F800802948D0F800902848006871
:10152000001D00F07FFB50B92548006890F82C1092
:101530000120884023490968814322480160681CD2
:10154000E0B9DEB100BF204948681D4909688860DC
:101550001B4982680968CA6019490968091D8268BF
:10156000516017490968091D8160174A14490968C3
:101570004A6111460968491C116018E07C1910483D
:1015800000684460BC4206D20D480168091D484607
:1015900000F06CFB0BE00A480168091D404600F0B2
:1015A00065FB0A480068844201D208480460BDE82F
:1015B000F087000024000020140000201800002004
:1015C00010000020280000204401002040000020DE
:1015D00010B5044600F064FB32480068401C3149F5
:1015E00008603148006840B92F4804600846006828
:1015F00001280DD100F080F90AE02C48006838B9C4
:1016000029480068C06AE16A884201D82648046017
:1016100027480068401C2649086000BF94F82C1039
:10162000012088402349096808432249086000BF17
:10163000E16A01EB8101204A02EB81014868A06068
:101640008268E260211D826851608160E16A01EB7D
:101650008101194A02EB81026261E16A01EB8101B9
:10166000154A52F82110491CE26A02EB8202124B21
:1016700043F8221000BF00BF00F024FB0B480068B5
:1016800078B100BF08480068C06AE16A884207D2A2
:101690004FF0805009490860BFF34F8FBFF36F8F41
:1016A00000BF10BD20000020100000202C000020F2
:1016B0003C000020280000209000002004ED00E005
:1016C00010B516E000F0ECFA0C48C068C468201DA4
:1016D00000F0A8FA0A480068401E09490860094855
:1016E0000068401E0749086000F0ECFA204600F050
:1016F0006CF8044800680028E4D110BD30010020D7
:10170000200000201C000020F0B587B00126002733
:10171000002408E012A0005D03A9085503A8005D9D
:1017200000B902E0641C102CF4DB00BF002510E0BF
:101730000D4F0E4800EB850000210B468022CDE9BD
:10174000001003A9384600F09DFB064606B902E0EA
:101750006D1C012DECDB00BF304607B0F0BD000072
:1017600049444C450000000049180008440000208E
:101770002DE9FF5F0746884616469946DDE90EAB20
:10178000B00000F045F9054675B14C2000F040F975
:1017900004462CB14C212046FEF798FD256304E059
:1017A000284600F09FFA00E0002454B100204B4688
:1017B00032464146CDE900ABCDE90240384600F063
:1017C00057F8204604B0BDE8F09F10B50446206BE2
:1017D00000F088FA204600F085FA10BD30B54FF4CD
:1017E0000053144800F007042CB1C01D20F007007E
:1017F000104C041B1B1B104C206000240E4D6C6011
:10180000C218083A22F007020C4C226000240B4D4B
:101810002D686C60094D2D682C600146541A4C608F
:10182000064C24680C60064D4C682C60054D4C68D5
:101830002C6030BD58010020540000205C000020C6
:10184000640000206000002000BFFFF739FF064859
:1018500000680128F9D94FF0805004490860BFF3AF
:101860004F8FBFF36F8FF0E79000002004ED00E092
:101870002DE9F05F81460E4617469A46DDF828802E
:101880000C9CB900A522206BFEF719FD781E216B78
:1018900001EB800B2BF0070B7EB1002507E0715D9B
:1018A00004F134004155705D00B902E06D1C102D4B
:1018B000F5D300BF002143200155B8F1050F01D336
:1018C0004FF00408C4F82C80201D00F0CCF904F17E
:1018D000180000F0C8F92461C8F10500A061646235
:1018E00052464946584600F013F920600B9808B15B
:1018F0000B980460BDE8F09F10B5002407E004EBEE
:1019000084010F4A02EB810000F0A0F9641C052C51
:10191000F5D30C4800F09AF90B4800F097F90B4802
:1019200000F094F90A4800F091F90A4800F08EF9A5
:1019300004480949086004480849086010BD0000CF
:1019400090000020F4000020080100201C0100206D
:101950003001002044010020140000201800002065
:1019600010B50146164800E0006803688B42FBD3BF
:101970000246436813448B4204D143684C682344B5
:10198000436001460A464B6813440468A34211D1E0
:101990000C4C03682468A34208D04B680468646850
:1019A00023444B6003681B680B6005E0054B1B6814
:1019B0000B6001E003680B60884200D0016010BD3D
:1019C000540000205C00002009480068006808B945
:1019D000012000E0002020B14FF0FF3005490860F1
:1019E00005E003480068C068006802490860704765
:1019F000140000204000002000BFBF2080F31188A9
:101A0000BFF34F8FBFF36F8F00BF00BFFEE7000033
:101A10002DE9F04704464FF00009DCB114F1090F3D
:101A200001D9012000E0002098B9083404F0070033
:101A300080B104F00700C0F10808C8F1FF30A042EF
:101A400001D2012000E0002008B9444402E0002453
:101A500000E0002400F0C0F92848006808B9FFF74A
:101A6000BDFE012000EBE470002841D0002C3FD0E7
:101A70002348006884423BD8224E3046056801E086
:101A80002E462D686868A04202D228680028F7D147
:101A90001A48006885422BD0306800F10809286890
:101AA00030606868001B102807D92F196868001B70
:101AB00078606C6030683860376011496868096820
:101AC000081A0F490860084600680F4909688842EB
:101AD00003D20B4800680C490860686840F0004079
:101AE00068600020286009480068401C07490860B9
:101AF00000F0B4FA4846BDE8F08700005C00002022
:101B000060000020540000206400002068000020D5
:101B1000001F4FF080730360001F21F0010303607A
:101B2000001F034B03601438026020387047000028
:101B3000F919000817B583B0144600BF1E480068A5
:101B400040F480701C49086000BF00BF1B4800685B
:101B500040F400401949086000BF9DF810008DF85E
:101B600004009DF811008DF805009DF812008DF815
:101B700006008DF808409DF80F008DF80A009DF8CA
:101B80000E008DF80900BDF80C00C0B28DF80B00F6
:101B90006A4600210A48FEF7D9FD02AA002108483A
:101BA000FEF7D4FC00BF0448006820F480700249AE
:101BB000086000BF06B010BD0070004070380240E1
:101BC0000028004000BF15480068C0F305401449D4
:101BD000087300BF11480068C0F30620487300BFB7
:101BE0000E48006800F07F00887300BF0B48406813
:101BF000C0F34230087100BF0848406800F03F0061
:101C0000887100BF05484068C0F30420487100BFD8
:101C100002484068C0F30740C87170470028004080
:101C20008000002001460A69D1E901309860D1E9BD
:101C3000010358605068884201D1886850600020D4
:101C400008611068401E10601068704700F10801BC
:101C500041604FF0FF31816000F10801C160016116
:101C600000210160704700210161704710B50246F4
:101C70000B685C1C0CB9106907E002F1080000E079
:101C80004068446824689C42FAD944684C604C68B7
:101C9000A160886041600A611468641C146010BD12
:101CA00000BFBF2080F31188BFF34F8FBFF36F8F4A
:101CB00000BF03480068401C0149086070470000ED
:101CC0005000002006480068401E0549086008468C
:101CD000006820B9002080F3118800BF00BF704762
:101CE0005000002070B506463546E6B1083D2C464A
:101CF0006068C00FB8B12068A8B9606820F00040E3
:101D0000606000F069F8084960680968084406499D
:101D100008602046FFF724FE04480068401C034981
:101D2000086000F09BF970BD600000206C0000208E
:101D300000204FF0E02108618861064800684FF4F8
:101D40007A71B0FBF1F0401E4FF0E02148610720AE
:101D5000086170470000002070B50446002544B1BA
:101D600000F03AF800212046FFF7CCFB00F076F9AE
:101D700005463DB94FF0805003490860BFF34F8FCF
:101D8000BFF36F8F70BD000004ED00E010B5FFF7EA
:101D9000BBFC0446012C14D100BFBF2080F3118886
:101DA000BFF34F8FBFF36F8F00BF4FF0FF30064977
:101DB000086001200549086000200549086000F01E
:101DC00047F80448006810BD400000202C000020A7
:101DD000240000204800002002480068401C0149FF
:101DE000086070474C0000201448006818B10120BA
:101DF0001349086021E000201149086000BF114824
:101E00000068B0FA80F0C0F11F0100BF01EB810251
:101E10000D4B03EB820042685268426000F10802F9
:101E20004368934201D1C26842604268D268074B5E
:101E30001A6000BF00BF1846006870474C000020C1
:101E40003400002028000020900000201000002016
:101E500010B50A48006840F47F0008490860084649
:101E6000006840F07F400860FFF762FF00200449EF
:101E70000860FEF7A7F9002010BD000020ED00E08B
:101E8000500000202DE9FC5F06460F46904699461B
:101E9000DDE90CAB4B46424639463046CDE900AB56
:101EA000FFF766FC054625B12846FFF791FB0124A4
:101EB00001E04FF0FF342046BDE8FC9F2DE9F041E2
:101EC00000275B48006800287DD15A480068451CFF
:101ED0005848056095B900BF5748D0F8008057486A
:101EE0000068554908605548C0F8008054480068AB
:101EF000401C53490860FFF767FD00BF5148006868
:101F000085427DD300BF4C480068006808B90120B5
:101F100000E0002020B14FF0FF304A4908606EE039
:101F200045480068C068C4686668B54202D2454842
:101F3000066064E000BF6069D4E902128A60D4E9F7
:101F400002214A60211D42688A4201D1E168416054
:101F5000002262610168491E016000BFA06AA0B151
:101F600000BFA06AD4E907128A60D4E907214A6059
:101F700004F1180142688A4201D1216A41600022BD
:101F8000A2620168491E016000BF00BF94F82C10D6
:101F9000012088402C49096808432B49086000BF8C
:101FA000E16A01EB8101294A02EB81014868A060E6
:101FB0008268E260211D826851608160E16A01EB04
:101FC0008101224A00E02BE002EB81026261E16ABA
:101FD00001EB81011D4A52F82110491CE26A02EB13
:101FE00082021A4B43F8221000BF00BF1849E06A72
:101FF0000968C96A884286D9012784E700E000BFE2
:1020000013480068C06A00EB8000104951F82000B6
:10201000012800D901270F48006800B1012704E01A
:102020000D480068401C0C4908603846BDE8F08146
:102030004C00002024000020140000201800002084
:1020400038000020400000202800002090000020E0
:102050001000002034000020300000202DE9F04165
:1020600000240027FFF71CFE002552480068401E90
:10207000504908600846006800286ED14E48006844
:1020800000286AD064E04D48C068C46800BFA06AF8
:10209000D4E907128A60D4E907214A6004F11801E3
:1020A00042688A4201D1216A41600022A26201682D
:1020B000491E016000BF00BF6069D4E902128A6056
:1020C000D4E902214A60211D42688A4201D1E168B7
:1020D0004160002262610168491E016000BF00BFCB
:1020E00094F82C1001208840354909680843344988
:1020F000086000BFE16A01EB8101324A02EB810115
:102100004868A0608268E260211D82685160816039
:10211000E16A01EB81012B4A02EB81026261E16A13
:1021200001EB8101274A52F82110491CE26A02EBB7
:102130008202244B43F8221000BF00BF2249E06A0C
:102140000968C96A884203D90120204941F825005D
:102150001A48006810B9012001E026E0002000289C
:1021600091D00CB1FFF730FC194806686EB100BF82
:10217000FFF7A4FE18B10120144941F82500761E8E
:10218000002EF5D1002012490860104850F82500B3
:1021900058B1012700BF0C48006838070D49086096
:1021A000BFF34F8FBFF36F8F00BFFFF78BFD384634
:1021B000BDE8F0814C000020200000201C01002020
:1021C0002800002090000020100000203400002093
:1021D0003000002004ED00E00000000000000000DE
:1021E00001020304060708090000000001020304BD
:1021F0005F6C697374006C69737420616C6C20632C
:102200006F6D6D616E6400002822000800000020E0
:1022100080000000F4120008A822000880000020BE
:10222000D8240000041300080024F400000000007B
:10223000000000000000000000000000000000009E
:10224000000000000000000000000000000000008E
:10225000000000000000000000000000000000007E
:10226000000000000000000000000000000000006E
:102270000400000000000000AAAAAAAA00000000B2
:10228000000000000000000000000000000000004E
:102290000000000000000000F0210008F621000806
:0822A000C6E533B43113000858
:040000050800018965
:00000001FF
